:020000040000FA
:040000006E303A28FC
:040004000034003490
:08000800A000030EA100831209
:100010008B1C32288B1032181428B21C3228643002
:10002000010203183128182800001628172818285C
:1000300019281A281B281C281D281E281F283210A2
:10004000B214A810031005190314AA0DA90DA80DC8
:10005000B10B322832152A08AF002908AE00280853
:10006000AD00B21081010B11210E8300A00E200EF5
:02007000090085
:0C007400203084008001840A80300402E7
:10008000031C3C281230B100912183160C308505E9
:1000900087018312850187010730990000309A009B
:1000A000103083168E008312603083168F00831207
:1000B0000030831691009F008312C83083168100A0
:1000C000831231309000003083168C008312103080
:1000D0008B00B12181018E018F010B118B100B1050
:1000E0008C018B178220321998207321B40B802841
:1000F000031085190314BA0DF0303A0203191A21BE
:10010000B22172286400321808000B1D08000B1180
:10011000B21032141230B100051D93283314831627
:10012000011383120800331083160117831208008D
:1001300032110130B7008B132030370783169B0034
:100140001C141A088312A400A500C030A5061030A4
:10015000370783169B001C141A088312A300003073
:10016000370783169B001C141A088312A2008B17F2
:10017000331CC02822090339A200A309A409A50938
:1001800022082D02031D142923082E02031D142901
:1001900024082F02031D142901303702031DD5281E
:1001A0003E18D5283E143F14992102303702031D12
:1001B000DE28BE18DE28BE143F149C21033037020F
:1001C000031DE7283E19E7283E153F149F21043000
:1001D0003702031DF028BE19F028BE153F14A221D6
:1001E00005303702031DF9283E1AF9283E163F1440
:1001F000A52106303702031D0229BE1A0229BE16A8
:100200003F14A82107303702031D0B293E1B0B2981
:100210003E173F14AB2108303702031D1429BE1BC3
:100220001429BE173F14AE21B70A0930370203184C
:1002300008009B280130B600B400B500B700850166
:100240008701B2138220B40B3629031085190314D9
:10025000BA0DF0303A0203195D29B51F8501B51FAB
:100260008701B50B36299630B5006721321D22294A
:100270003211331C40292D090339AD00AE09AF09F5
:100280002F1CB2132F1C2229B21B22292E1822291F
:10029000B2178B1320303707BC002F08BB007C211E
:1002A00010303707BC002E08BB007C210030370718
:1002B000BC002D08BB007C218B1785018701B70A84
:1002C000B60109303702031C2229B1210800370882
:1002D000B6080319B6000319080011308500133061
:1002E0008700B60308003F1C08003F101030BC0018
:1002F0003E08BB007C2108008B133B0883161C15AD
:100300009A0083123C0883169B0055309D00AA304A
:100310009D009C1464009C188A291C1183128B1761
:100320000800831610309B001C141A088312BE00AC
:1003300008000130BE0008000230BE000800043092
:10034000BE0008000830BE0008001030BE000800E3
:100350002030BE0008004030BE0008008030BE00E3
:10036000080008008F08031908008F0107303E05B8
:100370000319AA2A02303E05031D51105408EB3C14
:10038000031805125118C729D40BD229CC29D4033C
:100390005408C83C031CD2290516F530D400510876
:1003A000013AD10002303E05031DD1105508E63C4C
:1003B00003188512D118DF29D50BEA29E429D503C2
:1003C0005508B93C031CEA298516F030D5005108C0
:1003D000023AD10002303E05031D51115608DC3CA3
:1003E000031805105119F729D60B022AFC29D60348
:1003F0005608B63C031C022A0514E630D600510804
:10040000043AD10002303E05031DD1115708F03CDB
:1004100003188510D1190F2AD70B1A2A142AD703CB
:100420005708D73C031C1A2A8514FA30D700510804
:10043000083AD10002303E05031D51125808E03C35
:1004400003188710511A272AD80B322A2C2AD803CE
:100450005808C13C031C322A8714EA30D8005108DE
:10046000103AD10006303E05031DD1125908D43C84
:1004700003180711D11A3F2AD90B4A2A442AD90353
:100480005908A73C031C4A2A0715DE30D900510839
:10049000203AD10006303E05031D51135A08BF3CD7
:1004A00003180710511B572ADA0B622A5C2ADA0359
:1004B0005A089C3C031C622A0714C930DA00510810
:1004C000403AD10006303E05031DD1135B08D73CEE
:1004D00003188712D11B6F2ADB0B7A2A742ADB03DD
:1004E0005B08BE3C031C7A2A8716E130DB0051080A
:1004F000803AD10006303E05031D52105C08F13CE5
:10050000031807125218872ADC0B922A8C2ADC0364
:100510005C08CF3C031C922A0716FB30DC00520813
:10052000013AD20006303E05031DD2105D08E93CB9
:1005300003188711D2189F2ADD0BAA2AA42ADD03EB
:100540005D08B23C031CAA2A8715F330DD0052086F
:10055000023AD20018303E050319FA2ABE1DB62A07
:1005600054083C3C031CB62A85018701D40B0800C3
:10057000D0034630D4000B305002031DC02A0516AC
:100580000A305002031DC52A851609305002031D8A
:10059000CA2A051408305002031DCF2A85140730DB
:1005A0005002031DD42A871406305002031DD92A95
:1005B000071505305002031DDE2A071404305002CF
:1005C000031DE32A871603305002031DE82A07168D
:1005D00002305002031DED2A871501305002031D21
:1005E000F12A12305002031C0800850187010C30EB
:1005F000D000080020303E050319442BD40B052BF6
:100600000508103A85008230D400D50B0C2B050864
:10061000203A85007D30D500D60B132B0508013A12
:1006200085007330D600D70B1A2B0508023A8500D7
:100630008730D700D80B212B0708023A8700773084
:10064000D800D90B282B0708043A87006B30D90053
:10065000DA0B2F2B0708013A87005630DA00DB0B44
:10066000362B0708203A87006E30DB00DC0B3D2B71
:100670000708103A87008830DC00DD0B442B0708A0
:10068000083A87008030DD0040303E050319BB2B5F
:100690005408E63C03180512D40B6A2B0516F030FB
:1006A000D4002130DE070318682BB130D507FA30AB
:1006B000D607C830D7076430D8079630D907BE3080
:1006C000DA07AA30DB079A30DC07C430DD076A2B73
:1006D0008030BE005508823C03188512D50B732B61
:1006E00085168C30D5005608653C03180510D60BCE
:1006F0007C2B05146F30D6005708913C03188510E9
:10070000D70B852B85149B30D7005808D73C03188E
:100710008710D80B8E2B8714E130D8005908503C35
:1007200003180711D90B972B07155A30D9005A080F
:10073000873C03180710DA0BA02B07149130DA005E
:100740005B08BD3C03188712DB0BA92B8716C7304B
:10075000DB005C08703C03180712DC0BB22B071699
:100760007A30DC005D08A73C03188711DD0BBB2B3A
:100770008715B130DD0080303E050319C22B85019D
:060780008701DE01080004
:084000000B000300060009009B
:02400E00CC33B1
:10420000010003000300030003000200020002009B
:1042100002000000000000000000FF00FF00FF009F
:10422000000000000000000000000000000000008E
:104230000000C000C000C000C000FF00FF00FF0081
:104240000100C300F300CF00FF00C300F300CF0064
:10425000FF00C300F300CF00FF00FF00FF00FF00DE
:10426000FF00FF00FF00FF00FF00FF00FF00FF0056
:10427000FF00FF00FF00FF00FF00FF00FF00FF0046
:10428000FF00FF00FF00FF00FF00FF00FF00FF0036
:10429000FF00FF00FF00FF00FF00FF00FF00FF0026
:1042A000FF00FF00FF00FF00FF00FF00FF00FF0016
:1042B000FF00FF00FF00FF00FF00FF00FF00FF0006
:1042C000FF00FF00FF00FF00FF00FF00FF00FF00F6
:1042D000FF00FF00FF00FF00FF00FF00FF00FF00E6
:1042E000FF00FF00FF00FF00FF00FF00FF00FF00D6
:1042F000FF00FF00FF00FF00FF00FF00FF00AA001B
:00000001FF
